:10000000020C647DA37C08ED1D70011C144C70F77C
:0F001000EF1F70011E144E70EA22AE07020C7033
:10002300020BF04391405392BF53914F53924F228F
:10003B000205B8E5312425F8E60531227822300790
:10004B00027825E475F00112058202039A2000EB79
:10005B007F2ED2008018EF540F2490D43440D4FF5D
:10006B0030040BEF24BFB41A0050032461FFE532B8
:10007B00600215320535E5357002053430070D7811
:10008B0022E475F001120582EF02053A02001A74A0
:10009B0003D2078003E4C207F5318B228A2389241C
:1000AB00E4F532F534F535E53260077F201200793F
:1000BB0080F57533FFC201C200C202C203C205C282
:1000CB0006C208120047FF700D3007057F001200B3
:1000DB008AAF35AE3422B4255FC2D5C204120047B5
:1000EB00FF24D0B40A00501A75F00A783230D505C7
:1000FB0008B6FF0106C6A426F620D5047002D2036B
:10010B0080D924CFB41A00EF5004C2E5D204020206
:10011B008AD20180C6D20080C0D20280BCD2D580E8
:10012B00BAD20580B47F201200792002077401B582
:10013B00320040F112003EFF1200790200B2D208E9
:10014B00D206809512003EFB12003EFA12003EF9D9
:10015B004A4B7006795B7A037BFF20022EE53260F7
:10016B002A7E008E827583001203B360060EEE6545
:10017B003370F0C2D5EBC0E0EAC0E0E9C0E0EE12AC
:10018B0002D1D0E0F9D0E0FAD0E0FB12039AFF6085
:10019B00AAEBC0E0EAC0E0E9C0E0120079D0E024AD
:1001AB0001F9D0E03400FAD0E0FBE5330460DCD594
:1001BB0033D980877BFF7A0279CDD202809C79106C
:1001CB0080027908C206C2088008D2D5790A800459
:1001DB00790AC2D5E533047002F533E4FAFDFEFF6C
:1001EB0012003EFC7B0820011312003EFD7B1030F9
:1001FB00000A12003EFE12003EFF7B20EC3382D53C
:10020B0092D55013C3E43000069FFFE49EFEE4201A
:10021B0001039DFDE49CFCE4CBF8C201EC700CCF18
:10022B00CECDCCE824F8F870F38017C3EF33FFEE94
:10023B0033FEED33FDEC33FCEB33FB994002FB0F4C
:10024B00D8E9EB300105F8D0E0C448B201C0E00AB0
:10025B00EC4D4E4F78207B0070C2EAB5330040BCAA
:10026B00C0E01202D3D0F0D0E0200104C4C0E0C43F
:10027B00B201C0F0120062D0F0D5F0EB0200B21266
:10028B000592014F5301C95801204C011C4201CD6D
:10029B004F01D54401D54901354301DB5501BF461B
:1002AB0001BF4501BF47037B5001242D01282E01BF
:1002BB004B2B012C2301492003642A00E448000046
:1002CB0001433F3F3F00790AA2D5200314300509B3
:1002DB00B910020404B9080104A2D520060250018A
:1002EB00042002689202B532005034C0E07F203007
:1002FB0003197F30A20272067205500F12032AC235
:10030B0002C206C205C2087F30800F300503E9C068
:10031B00E0120079300503D0E0F9D0E0B532CC30F3
:10032B0005177F30B9100C1200797F583004077F06
:10033B00788003B908031200793002057F2D020083
:10034B00797F202008F87F2B2006F322920280CFA2
:10035B00286E756C6C2900D20112003E3001F8C278
:10036B0001783230D50108F60200E42D504349588C
:10037B0012003E2403B405004001E490037693126F
:10038B00006A743A12006AD2037532040201C9BBC7
:10039B00010689828A83E0225002E722BBFE02E338
:1003AB002289828A83E49322BB010CE58229F582A0
:1003BB00E5833AF583E0225006E92582F8E622BB75
:1003CB00FE06E92582F8E222E58229F582E5833AE9
:1003DB00F583E49322BB0110E58229F582E5833A8C
:1003EB00F583E0F5F0A3E0225009E92582F886F0C9
:1003FB0008E622BBFE0AE92582F8E2F5F008E222C4
:10040B00E5832AF583E993F5F0A3E9932275F008C8
:10041B00758200EF2FFFEE33FECD33CDCC33CCC541
:10042B008233C5829BED9AEC99E58298400CF5825C
:10043B00EE9BFEED9AFDEC99FC0FD5F0D6E4CEFBCE
:10044B00E4CDFAE4CCF9A88222B800C1B90059BABC
:10045B00002DEC8BF084CFCECDFCE5F0CBF97818EA
:10046B00EF2FFFEE33FEED33FDEC33FCEB33FB10E4
:10047B00D703994004EB99FB0FD8E5E4F9FA2278FE
:10048B0018EF2FFFEE33FEED33FDEC33FCC933C910
:10049B0010D7059BE99A4007EC9BFCE99AF90FD81A
:1004AB00E0E4C9FAE4CCFB2275F010EF2FFFEE333A
:1004BB00FEED33FDCC33CCC833C810D7079BEC9A79
:1004CB00E899400AED9BFDEC9AFCE899F80FD5F002
:1004DB00DAE4CDFBE4CCFAE4C8F922EB9FF5F0EAC1
:1004EB009E42F0E99D42F0E89C45F022E8600FEC5B
:1004FB00C313FCED13FDEE13FEEF13FFD8F122BB7C
:10050B00010DE58229F582E5833AF5830205595001
:10051B0007E92582F802054CBBFE07E92582F802A4
:10052B000565E58229F582E5833AF583020572BB01
:10053B00010689828A83F0225002F722BBFE01F367
:10054B0022E6FB08E6F908E6FA08E6CBF822E0F823
:10055B00A3E0F9A3E0FAA3E0FB22E2FB08E2F9082F
:10056B00E2FA08E2CBF822E493F8740193F97402EF
:10057B0093FA740393FB22FAE6FB0808E6F925F0DD
:10058B00F618E6CA3AF622D083D082F8E4937012BA
:10059B00740193700DA3A393F8740193F582888370
:1005AB00E4737402936860EFA3A3A380DFC0E0C081
:1005BB0083C082C0D075D000C002C004C005C00685
:1005CB00C00730D854C2D8AFDAC3EF9448748094C4
:1005DB00804015E50F2517F517E50E3516F5168531
:1005EB0017EAE516F5FA8031E5DA5411602B853EF2
:1005FB0036853F37AFFA753E008F3FE53FFEADEADC
:10060B007C00E42DF53FEC3EF53EC3E53F9537F519
:10061B0017E53E9536F516D20930D954C2D9AFDB62
:10062B00C3EF9448748094804015E5112519F51992
:10063B00E5103518F5188519EBE518F5FB8031E554
:10064B00DB5411602B854038854139AFFB75400079
:10065B008F41E541FEADEB7C00E42DF541EC3EF521
:10066B0040C3E5419539F519E5409538F518D20A9F
:10067B0030DA54C2DAAFDCC3EF9448748094804014
:10068B0015E513251BF51BE512351AF51A851BEC21
:10069B00E51AF5FC8031E5DC5411602B85423A8577
:1006AB00433BAFFC7542008F43E543FEADEC7C0052
:1006BB00E42DF543EC3EF542C3E543953BF51BE5D5
:1006CB0042953AF51AD20B30DB61ADBA43BA80C210
:1006DB00DB90FD54E0C39448748094804016E5157C
:1006EB002509F509E5143508F508A3E509F0E50832
:1006FB00A3F0803590FD54E05411602D85443C856A
:10070B00453D90FD56E0754400F545FE90FD55E0E6
:10071B007A002400F545EA3EF544C3E545953DF5E1
:10072B0009E544953CF508D20C8DBA30DF02C2DFE7
:10073B00D007D006D005D004D002D0D0D082D08341
:10074B00D0E0328B2B8A2C892DEF640160030208D9
:10075B00B7754601F547F548F549F54AF54BF54CA4
:10076B00FFEFC3948074809480500F74802FF582B8
:10077B00E43400F583E4F00F80E7E4FFEFC39480EB
:10078B0074809480500F74002FF582E43400F5834D
:10079B00E4F00F80E7AB2BAA2CA92D12039AFFE5EF
:1007AB0098543F4FF598EF64C06008EF64406003C6
:1007BB0002086690000212050A7F007E607D547C61
:1007CB00001204548F318E308D2F8C2EE4FFFE7D62
:1007DB0001FCAB31AA30A92FA82EC31204E64003AB
:1007EB007FFF22C3E49531F531E49530F530740188
:1007FB00952FF52FE4952EF52EAB2BAA2CA92D902A
:10080B0000011203B364027026538EEF438E015323
:10081B008EF7438E04AF31AE30AD2FAC2E7808126D
:10082B0004F78FD68531D753AFFB438E108066C24A
:10083B008E538EFE5389BF5389CF438E40AF31AE5B
:10084B0030AD2FAC2E78081204F78F8D85318BC20B
:10085B00AB5389BF538FFDD28E803AAB2BAA2CA9F9
:10086B002D12039AFF7E0070149000081203B364DC
:10087B00017005438E20801D538EDF8018EF64803E
:10088B004E70129000081203B36401700543878009
:10089B00800353877FAB2BAA2CA92D900007120343
:1008AB00B37004C29C8002D29C7F00227FFF22ADDA
:1008BB0007ED64047021C2DEF5F9F5E912039AFF26
:1008CB00E5D954F14FF5D99000041203B3640160DC
:1008DB000302099AD2DE22ED70279000011203B3B6
:1008EB00FFE5F2543F4FF5F29000021203E0F50FD3
:1008FB0085F00EC209850E16F5178517EAE516F574
:10090B00FAED640170279000011203B3FFE5F35475
:10091B003F4FF5F39000021203E0F51185F010C282
:10092B000A851018F5198519EBE518F5FBED64022E
:10093B0070279000011203B3FFE5F4543F4FF5F419
:10094B009000021203E0F51385F012C20B85121A08
:10095B00F51B851BECE51AF5FCED6403703143BA0E
:10096B00809000011203B3FF90FD57E0543F4FF00E
:10097B009000021203E0F51585F014C20C851408E3
:10098B00F50990FD55E509F0E508A3F053BA7F2270
:10099B00EF701FEC5403C4F854F0C8E4C4540F4870
:1009AB00FFE5F254CD4FFBEC5404C3134BF5F28D22
:1009BB00FA22EF6401701FEC5403C4F854F0C8E43E
:1009CB00C4540F48FFE5F354CD4FFBEC5404C31351
:1009DB004BF5F38DFB22EF6402701FEC5403C4F84C
:1009EB0054F0C8E4C4540F48FFE5F454CD4FFBEC6E
:1009FB005404C3134BF5F48DFC22EF6403702843AE
:100A0B00BA80EC5403C4F854F0C8E4C4540F48FF44
:100A1B0090FD57E054CD4FFBEC5404C3134BF090B7
:100A2B00FD56EDF053BA7F22E4F523752480F525AE
:100A3B00FB7A007922FF1208BAE4F523F524F52599
:100A4B00FB7A0079227F011208BAE4F52375243A68
:100A5B00752598FB7A0079227F021208BA7523C09C
:100A6B00E4F524F525FB7A0079227F031208BA7589
:100A7B0022087526017B007A0079227F041208BABE
:100A8B00E4FBFD7F04120ABFE4FB7D42FF120ABFA9
:100A9B00E4FB7D117F01120ABFE4FB7D4D7F021247
:100AAB000ABFE4FB7D427F03120ABF7DF47C017F0A
:100ABB000302099BEBF582758300D3940374809436
:100ACB00805030E582700553B77FC2BFE582640169
:100ADB004583700553B77FD2BFE5826402458370AF
:100AEB000543B780C2BFE58264034583700543B7F6
:100AFB0080D2BFEF14601114601214601314601DC8
:100B0B00240470248DDA80208DDB801C8DDC801812
:100B1B0043BA8090FD54EDF053BA7F800BED540136
:100B2B00FFE5D954FE4FF5D97F0022120026120C97
:100B3B003B120A33D2AF751C80C20D7BFF7A0C7946
:100B4B007A1200A07F017E00120003300A11C20A44
:100B5B007BFF7A0C799C8518258519261200A00538
:100B6B001DE51D540F640F70DB300D11151CD3E503
:100B7B001C9408748094805013C20D800F051CC305
:100B8B00E51C94F8748094804002D20DE51CFD7C2A
:100B9B0000E4FF12099B80ACEFFBD39401748094AB
:100BAB00805009EB7004C2AC8002D2ACEDFF7E002A
:100BBB00D39403748094805029EF700553B7EFC220
:100BCB00BCEF64014E700553B7EFD2BCEF64024E1D
:100BDB00700543B710C2BCEF64034E700543B710EA
:100BEB00D2BC7F0022C0E0C083C082C0D075D000D1
:100BFB00C007309828C298E54C7022C3E54A948010
:100C0B00748094804003754A00AF4A054A74002FE4
:100C1B00F582E43400F583E599F0754B05309905C1
:100C2B00C299754900D007D0D0D082D083D0E032A2
:100C3B007522407523017527007526C27525017530
:100C4B002400752901E4F52AFB7A0079227F011231
:100C5B00074E7D017F01020BA3787FE4F6D8FD756B
:100C6B00814C020B368F99754901E54970FC225373
:100C7B0054433841384B363444342050434120548C
:100C8B006573742050726F6772616D6D65210D0A0B
:0E0C9B0000436170747572653D25640D0A009A
:00000001FF
